:100000000C946B000C9488000C9488000C94E9020A
:100010000C9488000C9488000C9488000C94880040
:100020000C9488000C94821C0C9488000C9488001A
:100030000C9488000C94201A0C9488000C9488006E
:100040000C9488000C9488000C9488000C94880010
:100050000C94880007634236B79BD8A71A396856B4
:1000600018AEBAAB558C1D3CB7CC5763BD6DEDFDDA
:10007000753EF6177231BF000000803F0800000097
:10008000BE922449123EABAAAA2ABECDCCCC4C3E8D
:1000900000000080BEABAAAAAA3E00000000BF007C
:1000A0000000803F0000000000084178D3BB438778
:1000B000D1133D190E3CC3BD4282AD2B3E68EC828C
:1000C00076BED98FE1A93E4C80EFFFBE01C4FF7F11
:1000D0003F000000000011241FBECFE5D8E0DEBFC6
:1000E000CDBF11E0A0E6B0E0E0E6FAE402C0059082
:1000F0000D92A63EB107D9F713E0A6EEB1E001C01C
:100100001D92A334B107E1F70E94B8160C942F2575
:100110000C9400005D9BFECF8CB90895EF92FF9286
:100120000F931F937B018C0120E030E040E050E012
:1001300008C080EA9FE00197F1F72F5F3F4F4F4FD4
:100140005F4F2E153F054007510799F71F910F91FB
:10015000FF90EF900895EF92FF920F931F937B0112
:100160008C0120E030E040E050E007C085E38A9554
:10017000F1F72F5F3F4F4F4F5F4F2E153F05400761
:100180005107A1F71F910F91FF90EF90089588B349
:10019000806F88BB87B3806B87BB8DB18DB98DB104
:1001A00083658DB90895BC9A80E48DB908958FB99F
:1001B000779BFECF0895779BFECF8FB190E0089597
:1001C000949A64E670E080E090E00E948E0094983B
:1001D00080E090E00895C498880F8E778FB9779B60
:1001E000FECF6FB9779BFECFC49A0895C498880F4D
:1001F0008E7780688FB9779BFECF1FB8779BFECF35
:100200008FB1C49A90E008950F931F93182F062F73
:10021000682F66956695669580E00E94EB00602FDA
:10022000812F0E94EB001F910F910895682F80E0AD
:100230000E94040108951F93182F682F66956695F4
:10024000669580E00E94EB00812F0E94F60090E00E
:100250001F9108950F931F93082F162F0E941B01C3
:1002600010951823612F802F0E9404011F910F9178
:1002700008950F931F93082F162F0E941B01182B10
:10028000612F802F0E9404011F910F91089561E05A
:1002900089E00E94390108958F929F92BF92CF9278
:1002A000DF92EF92FF920F931F93CF93DF93CDB71F
:1002B000DEB721970FB6F894DEBF0FBECDBFF82E84
:1002C0008B016A0149016FE786E00E9404016FE734
:1002D00087E00E9404010E94470185E00E941B0103
:1002E00086FFFBCF60E081E00E94040189E20E946A
:1002F0001B01B82E60E289E20E9404019092E7019E
:100300008092E6011093E9010093E801D092EB019D
:10031000C092EA01F40114868BB780628BBFFCE0C7
:10032000FF1609F446C0FF1590F083E0F816C1F1FE
:100330008F1530F0FF2049F1E1E0FE16E9F42AC004
:10034000F7E0FF16F9F08BE0F816B1F42EC0E6E105
:10035000FE16B1F1EF1538F0F2E1FF1671F184E10C
:10036000F81651F40BC0E9E1FE1630F0FAE1FF1582
:1003700048F48EE1F816E1F119E104C15FE1C52E00
:1003800004E04BC04FE1C42E12C03FE1C32E00E099
:1003900090E044C027E1C22E01E190E110E03FC0AF
:1003A00097E1C92E07E094E0F9CF87E1C82E05E078
:1003B000FACF0FE1C02E05E030C01FE1C12EECCF17
:1003C0008FE00E941B0182958F7090E0909581953F
:1003D0009F4FAA2797FDA095BA2FF4018087918798
:1003E000A287B387BFE1CB2E06E094E014E017C0EC
:1003F0008FE00E941B0182958F7090E0909581950F
:100400009F4FAA2797FDA095BA2FF4018087918767
:10041000A287B387AFE1CA2E0DE394E012E08AE130
:1004200099830E941B01F0E4EF2EE822998186FD5A
:1004300005C060E48AE10E9439019981E0E2DE2E84
:10044000D92A006A602F86E00E940401612F8BE2A6
:100450000E94040111FD04C062E089E00E9439019C
:100460006F2D81E00E940401E091E601F091E70127
:1004700084858D21E9F364E089E00E9439016FE70A
:1004800086E00E9404016FE787E00E94040160E0BB
:1004900081E00E940401E091E601F091E701118101
:1004A000848585FF04C096858785892B8687E091A2
:1004B000E601F091E7018685C822C686E091E60153
:1004C000F091E7018685882329F1868580FF07C0A2
:1004D0008BE00E941B01F40185871AE103C0868529
:1004E00081FD18E0E091E601F091E701868582FF49
:1004F00002C017E10FC0868584FF04C00E94470137
:1005000015E108C0868583FF02C014E003C01123F3
:1005100009F414E6FEE1FF1619F086E1F81661F51C
:1005200085E00E941B01682F677081F0F40120852F
:100530003185428553858681978173E0880F991FA5
:100540007A95E1F70897860F911D0CC0F40120857C
:100550003185428553858681978163E0880F991F95
:100560006A95E1F7A0E0B0E0820F931FA41FB51FCA
:1005700080879187A287B387EE2021F460E48AE127
:100580000E942A018BB78F7D8BBF1092E7011092DA
:10059000E6011092E9011092E8011092EB0110922D
:1005A000EA016B2D89E20E940401812F90E02196DF
:1005B0000FB6F894DEBF0FBECDBFDF91CF911F9174
:1005C0000F91FF90EF90DF90CF90BF909F908F9012
:1005D00008951F920F920FB60F921124BF92CF92DF
:1005E000DF92EF92FF920F931F932F933F934F93BE
:1005F0005F936F937F938F939F93AF93BF93CF93AB
:10060000DF93EF93FF938091E6019091E701892BAF
:1006100009F453C18091E8019091E901892B09F413
:100620004CC18091EA019091EB01892B09F445C1FD
:1006300080E00E94F600B82E8093F0010091E60160
:100640001091E7018AE00E941B018F70F8018687F4
:10065000C090F101E090EF010091EE01F090F20105
:100660001BC186E00E941B01C82E87E00E941B016F
:10067000F82EFC20E091E601F091E70184858F29B6
:100680008487CF2DF0FE43C084E00E941B0160E40C
:10069000E62EE81AE091E601F091E7018481958168
:1006A00022813381821B930B2E2D30E028173907CE
:1006B00050F02481358182819381E22EE81A61E035
:1006C00086E00E94040100E01BC0E091E601F09189
:1006D000E7010280F381E02D8091E8019091E9012A
:1006E000E80FF91F608182E00E940401E091E601B9
:1006F000F091E701828193810196938382830F5F5A
:100700000E1519F761E087E00E9404010E2DC4FF69
:1007100017C060E187E00E94040162E886E00E9461
:100720000401E091E601F091E7018089882341F01E
:1007300062E082E20E94040160E080E00E94EB003F
:10074000C3FF28C0E091E601F091E7018189882389
:1007500019F48685882339F460E081E00E94040161
:10076000F4E0FF2A17C086858787E091E601F091C3
:10077000E701168661E089E00E940401E091E6014C
:10078000F091E7011782168287EFF82268E087E090
:100790000E940401CF2DD0E0CE018E709070892B85
:1007A00009F440C084E00E941B01E82E00E026C04E
:1007B000E091E601F091E70186819781D02ED394F4
:1007C00080349105C0F4068117818091EA019091EF
:1007D000EB01080F191F82E00E941B01F8018083C2
:1007E000E091E601F091E701868197810196978378
:1007F00086830D2D03C080E7818302C00E15C1F6EC
:1008000084E00E941B01E82EE091E601F091E701EF
:100810008181882311F4EE2049F66F2D6A7087E0FC
:100820000E940401C1FF0FC083E00E941B0180777A
:10083000803749F489E00E941B01082F682F64600B
:1008400089E00E940401C2FF18C060E286E00E94B5
:10085000040164E287E00E940401FFEDFF22E091C1
:10086000E601F091E70184858F7D8487E091E601C0
:10087000F091E701848584608487F5FE0DC060E215
:1008800087E00E940401E091E601F091E701818197
:10089000882311F481E0818383E00E941B0183FDA2
:1008A000E0CEC092F101E092EF010093EE01F092F0
:1008B000F2016B2D80E00E940401FF91EF91DF9126
:1008C000CF91BF91AF919F918F917F916F915F91E8
:1008D0004F913F912F911F910F91FF90EF90DF90DB
:1008E000CF90BF900F900FBE0F901F901895DC0116
:1008F000FB0140E02D91322F3F7022952F70832F06
:1009000090E08095909554E0880F991F5A95E1F7F3
:10091000382B3183822F90E08095909574E0880F7A
:10092000991F7A95E1F7282B20834F5F3296463046
:1009300009F780E090E00895FF920F931F93CF9303
:10094000DF93CDB7DEB72C970FB6F894DEBF0FBE9E
:10095000CDBFF82ECB018E010F5F1F4FB8010E9453
:100960007704982F882339F580E6F81689F420E07B
:1009700030E0B801FB01E20FF31F8081F901EA5E6C
:10098000FD4F80832F5F3F4F2C303105A1F0F2CF18
:1009900081E6F81681F420E030E0B801FB01E20FB7
:1009A000F31F8081F901E850FE4F80832F5F3F4F96
:1009B0002C30310599F7892F90E02C960FB6F894DA
:1009C000DEBF0FBECDBFDF91CF911F910F91FF9082
:1009D0000895FF920F931F93CF93DF938C01F62E10
:1009E0000E944701602F82E00E940401012F11271D
:1009F000602F82E00E9404016F2D82E00E940401BA
:100A000063E081E00E94040181E00E941B018823D1
:100A1000D9F7C2E2D2E000E005C082E00E941B01EB
:100A200089930F5F0F15C9F780E090E0DF91CF91B8
:100A30001F910F91FF900895DF92EF92FF920F9315
:100A40001F93CF93DF938C01D62E7A010E9447012A
:100A5000602F82E00E940401012F1127602F82E0A5
:100A60000E940401E70100E005C0699182E00E9454
:100A700004010F5F0D15C9F761E081E00E940401D8
:100A800085E00E941B0186FFFBCF60E081E00E94B1
:100A9000040180E090E0DF91CF911F910F91FF90D2
:100AA000EF90DF900895EF92FF920F931F93CF93F3
:100AB000DF93CDB7DEB72C970FB6F894DEBF0FBE2D
:100AC000CDBF98E1699F8001112400581F4F8136E6
:100AD00011F4045F1F4F7E010894E11CF11CB70163
:100AE000CA010E947704882329F4A7016CE0C80199
:100AF0000E941C0590E02C960FB6F894DEBF0FBE46
:100B0000CDBFDF91CF911F910F91FF90EF9008958E
:100B10000F931F93CF93DF938C010E944701C0E096
:100B2000D0E0F801EC0FFD1F608182E00E9404011B
:100B30002196CC30D105A9F769E181E00E9404013A
:100B400081E00E941B018823D9F70E941B01803499
:100B500009F48BE090E0DF91CF911F910F91089500
:100B6000EF92FF920F931F937B018C0167E005C00A
:100B70006F5F16950795F794E7948FEFE816F104E9
:100B80000105110509F0A0F7663130F065E1EFEFDE
:100B9000EE2EF12C012D112D8AE20E9404016E2D02
:100BA0008CE20E94040180E090E01F910F91FF9081
:100BB000EF9008951F936AE670E080E090E00E9455
:100BC000B00567E082E20E940401109204021092D4
:100BD0000502109210021092070210920602109263
:100BE00009021092080210920B0210920A0210924F
:100BF0000C0210920D0210920E0210920F0210922F
:100C0000110210921202109213021092140210920A
:100C10001502E0917100F091720080E58083E0910F
:100C20007100F0917200118282E090E090930902CD
:100C3000809308024091730050917400609171009C
:100C40007091720024E032E08EE10E944C01182F76
:100C5000882329F0813011F08E3109F410E060E032
:100C600081E00E940401812F90E01F910895CF93AD
:100C7000DF936EE08DE10E9404016091ED01C62FCB
:100C8000D0E0CC0FDD1FCC0FDD1FCB56DF4F6881CE
:100C900084E10E9404016A8185E10E94040160915F
:100CA000EC01C62FD0E0A3E0CC0FDD1FAA95E1F741
:100CB000CB58DF4F688189E10E9404016A818AE193
:100CC0000E9404016C818CE10E9404016E818DE11F
:100CD0000E94040180E090E0DF91CF91089584307C
:100CE00050F4643040F48093EC016093ED010E9475
:100CF000370680E001C085E290E008958091EC0124
:100D0000882331F08091ED01882311F080E004C048
:100D100060E080E00E946F0690E0089560E08FE15F
:100D20000E94040160E48FE10E94040164E170E02C
:100D300080E090E00E94AB0060E48FE10E942A0115
:100D400061E48EE10E94040163E08DE20E940401EF
:100D50006FE382E10E9404016FE383E10E940401DA
:100D600080E090E00895CF93DF93EC0163E081E1B0
:100D70000E942A01209749F0BE0180E090E00E9485
:100D80008E0063E081E10E94390180E090E0DF9114
:100D9000CF9108951F930E94E000182F882349F4F3
:100DA0000E948E06182F0E94370681E090E00E9474
:100DB000B306812F90E01F91089563E081E10E94C6
:100DC0002A01089562E081E10E9439010895DC0161
:100DD000FB0140E02D91322F3F7022952F70832F21
:100DE00090E08095909554E0880F991F5A95E1F70F
:100DF000382B3183822F90E08095909534E0880FD6
:100E0000991F3A95E1F7282B20834F5F32964630A1
:100E100009F780E090E008951F93162F0E94470184
:100E200066E181E00E94040165E070E080E090E00E
:100E30000E948E00E2E2F2E090E003C082E0819343
:100E40009F5F9117D9F760E081E00E94040180E084
:100E500090E01F910895FF920F931F93CF93DF931C
:100E60008C01F62E0E9447016BE581E10E9404018E
:100E7000E80100E005C0699182E00E9404010F5F73
:100E80000F15C9F76EE181E00E94040180E090E057
:100E9000DF91CF911F910F91FF900895FF920F93D3
:100EA0001F93CF93DF938C01F62E0E9447016BE5D1
:100EB00081E10E9404016AE181E00E940401E801ED
:100EC00000E005C0699182E00E9404010F5F0F15E8
:100ED000C9F760E081E00E94040180E090E0DF91CA
:100EE000CF911F910F91FF90089563E789E10E94D0
:100EF00004016DEA8BE10E9404016FEF8CE10E9416
:100F000004016EE18DE10E94040161E08EE10E9426
:100F1000040160E08FE10E94040168E089E00E9422
:100F2000040169E184E10E94040163E185E10E941A
:100F300004016BE581E10E94040166E081E20E9408
:100F4000040163E08DE20E94040163E082E20E94FA
:100F500004016FE383E10E94040180E090E00895C2
:100F6000EF92FF920F931F93CF93DF93F82E8B0195
:100F7000E42E67E082E20E94040166E970E080E00E
:100F800090E00E94B005E0917100F0917200F08253
:100F9000E0917100F0917200E182E0917100F091B6
:100FA0007200E80188819981AA81BB818283938341
:100FB000A483B583109204021092050210921002CD
:100FC0001092070210920602109209021092080273
:100FD00010920B0210920A0210920C0210920D0253
:100FE00010920E0210920F02109211021092120231
:100FF00010921302109214021092150286E090E0F3
:1010000090930902809308024091730050917400FC
:10101000609171007091720024E032E08CE00E94D7
:101020004C01082F882309F04BC085E00E941B016A
:1010300090E087709070892B11F00DE041C063E063
:1010400082E20E94040110920402109205021092A2
:1010500010021092070210920602109209021092DA
:10106000080210920B0210920A0210920C021092C7
:101070000D0210920E0210920F02109211021092A5
:101080001202109213021092140210921502109282
:10109000090210920802409173005091740060910F
:1010A00071007091720024E032E084E10E944C01F2
:1010B000082F882329F489E00E941B0183FF07E0A1
:1010C000802F90E0DF91CF911F910F91FF90EF90D3
:1010D0000895EF92FF920F931F93CF93DF93CDB7B5
:1010E000DEB722970FB6F894DEBF0FBECDBFF82E45
:1010F0008B01E22E88E1489FA001112440585F4FE8
:101100005A8349836AE670E080E090E00E94B0056F
:1011100081E6F81629F489819A810C969A8389834D
:101120000E944701109204021092050210921002D0
:101130001092070210920602109209021092080201
:1011400010920B0210920A0210920C0210920D02E1
:1011500010920E0210920F021092110210921202BF
:10116000109213021092140210921502E091710075
:10117000F091720089819A819183808382E090E06E
:10118000909309028093080240917300509174007B
:10119000609171007091720024E032E08BE00E9457
:1011A0004C01882329F44E2DB8018F2D0E94B007E1
:1011B00090E022960FB6F894DEBF0FBECDBFDF9150
:1011C000CF911F910F91FF90EF900895242F462FFC
:1011D00063EF71E00E94690890E00895EF92FF923A
:1011E0000F931F93CF93DF93E82EEB018A01F22E2A
:1011F0006AE670E080E090E00E94B0050E9447013E
:10120000109204021092050210921002109207022E
:1012100010920602109209021092080210920B021C
:1012200010920A0210920C0210920D0210920E02FD
:1012300010920F02109211021092120210921302D9
:101240001092140210921502A0917100B0917200D8
:10125000F8018CE001900D928150E1F78CE090E074
:10126000909309028093080240917300509174009A
:10127000609171007091720024E032E089E10E9477
:101280004C01882329F44F2DBE018E2D0E94B007FA
:1012900090E0DF91CF911F910F91FF90EF90089513
:1012A000FF920F931F93CF93DF93182F062FF42EE7
:1012B000E90160ED77E080E090E00E94B00567E032
:1012C00082E20E9404011092040210920502109220
:1012D0001002109207021092060210920902109258
:1012E000080210920B0210920A0210920C02109245
:1012F0000D0210920E0210920F0210921102109223
:101300001202109213021092140210921502E09130
:101310007100F09172001083E0917100F091720001
:10132000018382E090E0909309028093080240914B
:10133000730050917400609171007091720024E00C
:1013400032E08EE10E944C01813009F4E1C08091CD
:101350000C0290910D02A0910E02B0910F0208971D
:10136000A105B105C1F48AE10E941B0180FF13C0F1
:10137000E0917300F09174008081282F30E02F708D
:10138000307082958F7090E02817390711F488E04B
:1013900003C080E001C084E020910C0230910D0276
:1013A00040910E0250910F0290E0A0E0B0E0E09179
:1013B0007300F0917400281739074A075B0709F496
:1013C00089C080818F708083E0917300F0917400F8
:1013D000E081EE2309F499C0EA3009F098C0109238
:1013E000040210920502109210021092070210924D
:1013F0000602109209021092080210920B0210923B
:101400000A0210920C0210920D0210920E0210921B
:101410000F021092110210921202109213021092F7
:101420001402109215020F2D10E0A801BE01809148
:101430007100909172000E94CE21109309020093D6
:101440000802409173005091740060917100709196
:10145000720024E032E08EE10E944C01813009F4F8
:1014600057C080910C0290910D02A0910E02B09194
:101470000F020897A105B105C1F48AE10E941B0182
:1014800080FF13C0E0917300F09174008081282FD9
:1014900030E02F70307082958F7090E028173907F8
:1014A00011F488E003C080E001C084E020910C02C8
:1014B00030910D0240910E0250910F0290E0A0E099
:1014C000B0E0E0917300F0917400281739074A07E3
:1014D0005B0759F480818F708083E0917300F091F5
:1014E000740080818A7099F410C080818F7080832D
:1014F000E0917300F0917400E081EE2321F0EA3076
:1015000031F480E005C081E103C08CE001C089E0D6
:1015100090E0DF91CF911F910F91FF9008959B0173
:1015200040E1682F80EA0E94500990E00895FF9200
:101530000F931F93CF93DF93F82E8B0168EE73E028
:1015400080E090E00E94B00567E082E20E94040122
:1015500010920402109205021092100210920702DB
:1015600010920602109209021092080210920B02C9
:1015700010920A0210920C0210920D0210920E02AA
:1015800010920F0210921102109212021092130286
:101590001092140210921502E0917100F091720005
:1015A00082EA8083E0917100F0917200F182E09113
:1015B0007100F0917200E80188819981AA81BB8154
:1015C00082839383A483B58386E090E0909309029D
:1015D00080930802409173005091740060917100F3
:1015E0007091720024E032E08EE10E944C01813063
:1015F00009F451C080910C0290910D02A0910E024D
:10160000B0910F020897A105B105C1F48AE10E94CB
:101610001B0180FF13C0E0917300F0917400808182
:10162000282F30E02F70307082958F7090E028174F
:10163000390711F468E003C060E001C064E0209164
:101640000C0230910D0240910E0250910F02862F34
:1016500090E0A0E0B0E0281739074A075B0731F0B7
:10166000662311F481E217C08DE015C0E09173008C
:10167000F091740080818F708083E0917300F0910D
:101680007400E081EE2331F0EA3011F480E003C011
:1016900089E001C08CE090E0DF91CF911F910F9124
:1016A000FF900895FF920F931F93CF93DF93182F0E
:1016B000062FF42EE9010E94470160E872E080E005
:1016C00090E00E94B0056FE082E20E940401109257
:1016D000040210920502109210021092070210925A
:1016E0000602109209021092080210920B02109248
:1016F0000A0210920C0210920D0210920E02109229
:101700000F02109211021092120210921302109204
:10171000140210921502E0917100F0917200108392
:10172000E0917100F0917200018382E090E090936B
:1017300009028093080240917300509174006091F7
:1017400071007091720024E032E08EE10E944C0141
:10175000182F882309F472C0813009F46AC080917F
:101760000C0290910D02A0910E02B0910F02089709
:10177000A105B105C9F48AE10E941B0180FF14C0D4
:10178000E0917300F09174008081282F30E02F7079
:10179000307082958F7090E02817390711F488E037
:1017A00004C011E280E001C084E020910C0230917D
:1017B0000D0240910E0250910F0290E0A0E0B0E0C7
:1017C000281739074A075B0791F4E0917300F091FD
:1017D000740080818F708083E0917300F0917400B9
:1017E00080818A7011F41CE05EC019E05CC08091B9
:1017F0000A0290910B024F2D50E06091730070919E
:1018000074008417950708F04BC040910A0250916C
:101810000B02CE010E94CE2180910A0290910B0210
:1018200005C0FE01E80FF11D10828F5F8F15C8F310
:101830003AC04F2D50E060E670E032C080910A025D
:1018400090910B024F2D50E08417950721F1809164
:101850000A0290910B0260917300709174008417DA
:10186000950720F0CE010E94CE2113C040910A02BC
:1018700050910B02CE010E94CE2180910A029091DC
:101880000B0205C0FE01E80FF11D10828F5F8F155E
:10189000C8F31EE008C06091730070917400AC0141
:1018A000CE010E94CE21812F90E0DF91CF911F9138
:1018B0000F91FF9008959B0140E1682F80E30E9403
:1018C000520B90E00895FF920F931F93CF93DF93F5
:1018D000F82EEB018A010E947E06282F882309F04A
:1018E0008EC06AE670E080E090E00E94B0056FE094
:1018F00082E20E94040168E089E00E942A011092BD
:101900000402109205021092100210920702109227
:101910000602109209021092080210920B02109215
:101920000A0210920C0210920D0210920E021092F6
:101930000F021092110210921202109213021092D2
:10194000140210921502E0917100F0917200F08281
:10195000E0917100F091720080E78183E091710065
:10196000F091720088819981AA81BB8182839383DF
:10197000A483B583E0917100F0917200838192811C
:1019800089279481892795818927868387E090E03C
:10199000909309028093080281E0809315024091A0
:1019A00073005091740024E032E0BF018EE10E9488
:1019B0004C01282FF80110828823D1F480910C0269
:1019C00090910D02A0910E02B0910F020897A1050F
:1019D000B10511F02DE00CC088819981AA81BB81ED
:1019E0008093F3019093F401A093F501B093F60175
:1019F000E0917300F09174008081F8018083822F60
:101A000090E0DF91CF911F910F91FF900895AB016E
:101A1000BC0183E90E94630C90E008954F925F92AD
:101A20006F927F928F929F92AF92BF92CF92DF92EE
:101A3000EF92FF920F931F93CF93DF93CDB7DEB753
:101A400024970FB6F894DEBF0FBECDBFC82ED62E9A
:101A50004A010E947E06F82E882309F07DC16AE6BD
:101A600070E080E090E00E94B005F40180819181F7
:101A7000A281B38189839A83AB83BC8368E28AE1C4
:101A80000E94040168E089E00E942A015E01089436
:101A9000A11CB11CA4E06A2EA2E07A2EF0E2FD1592
:101AA00018F4FCE3FF2E58C11092040210920502B4
:101AB0001092100210920702109206021092090270
:101AC0001092080210920B0210920A0210920C025D
:101AD00010920D0210920E0210920F02109211023B
:101AE0001092120210921302109214021092150218
:101AF000C092040201E00093150263E082E20E94BA
:101B00000401E7E0EE2EED201D2D16951695169595
:101B1000EE20E9F06E2D6295607F6E298FE00E94C5
:101B200004011F5F87E0E81691F40093140287E038
:101B300090E0A0E0B0E080930C0290930D02A0939F
:101B40000E02B0930F0267E08FE00E940401E09163
:101B50007100F0917200C082E0917100F09172000A
:101B60009E2D905E8D2D8695869586958295807F9B
:101B7000980F918320E030E0412F50E00AC0A20F7F
:101B8000B31FF501E20FF31F8081FD0182832F5FF8
:101B90003F4F8A01A0917100B09172002417350760
:101BA00071F70E5F1F4F1093090200930802025055
:101BB000104040917300509174009301BD018EE17B
:101BC0000E944C01F82E80911402882309F456C01B
:101BD00040E050E070E01FC0E0917300F0917400AD
:101BE000E40FF51F6081262F30E087E090E0841B32
:101BF000950B02C0220F331F8A95E2F7872F90E0E2
:101C00004F5F5F4F042E02C0959587950A94E2F7C7
:101C1000282B2083762F80910A0290910B0248177F
:101C20005907D0F280910C0290910D02A0910E0202
:101C3000B0910F0220910A0230910B0240E050E077
:101C4000821B930BA40BB50B80930C0290930D0297
:101C5000A0930E02B0930F0280911102882371F0BD
:101C60002091110280911102295F90E0069669E0AF
:101C700070E00E94F021261B20931102FF2021F02A
:101C8000FAE1FF1609F068C019821A821B821C82D1
:101C9000EE2011F480E010C001501040E09173007C
:101CA000F09174009081F501E00FF11F0F5F1F4F5D
:101CB0008081892B808381E0E0917300F091740032
:101CC000BF01680F711D2501400E511E40E050E01C
:101CD00024E030E0201B310B08C0DB018D91BD01F9
:101CE000D2018D932D014F5F5F4F42175307ACF325
:101CF00020910C0230910D0240910E0250910F0282
:101D000088E290E08D199109AA2797FDA095BA2F36
:101D1000281739074A075B0719F07DE0F72E1CC02A
:101D2000BAE1FB1691F080910A0290910B02319773
:101D3000E80FF91F20818A81998189279B81892752
:101D40009C818927821731F407C080911102D80E37
:101D5000DE18A4CE6AE0F62E89819A81AB81BC811F
:101D6000F40180839183A283B38360E28AE10E94BD
:101D70002A018F2D90E024960FB6F894DEBF0FBE97
:101D8000CDBFDF91CF911F910F91FF90EF90DF902A
:101D9000CF90BF90AF909F908F907F906F905F900B
:101DA0004F900895AB01682F83E90E940E0D90E0DB
:101DB00008951F93CF93DF93182FEB010E947E06A7
:101DC000882311F0282F8FC06CE370E080E090E052
:101DD0000E94B00563E082E20E94040168E089E0AD
:101DE0000E942A0167E08FE00E9404011092040221
:101DF0001092050210921002109207021092060231
:101E0000109209021092080210920B0210920A021C
:101E100010920C0210920D0210920E0210920F02FC
:101E200010921102109212021092130210921402D8
:101E300010921502E0917100F0917200108381E020
:101E400090E0909309028093080281E0809315024C
:101E50004091730050917400609171007091720014
:101E600024E032E08EE10E944C01282F882371F497
:101E700080910C0290910D02A0910E02B0910F0280
:101E80004097A105B10589F02DE00FC08A3169F4B2
:101E900080910C0290910D02A0910E02B0910F0260
:101EA0004097A105B10509F420E080910A029091C4
:101EB0000B02029748F0E0917300F091740080816A
:101EC0009181998388830FC080910A0290910B02BF
:101ED000019739F4E0917300F09174008081888358
:101EE00002C018821982822F90E0DF91CF911F915A
:101EF00008952F923F924F925F926F927F928F92AE
:101F00009F92AF92BF92CF92DF92EF92FF920F9388
:101F10001F93CF93DF93CDB7DEB724970FB6F89416
:101F2000DEBF0FBECDBF182F7B016A013901802EA5
:101F30000E947E06282F882309F075C0B70182E52C
:101F40000E94D90E282F882309F06DC0F7018081E7
:101F500090E08F719070892B11F42FE164C01130E3
:101F600071F0113050F0123021F0133021F025E2E1
:101F70005AC004E905C008E903C003E901C002E949
:101F800088E8898310E0EE24FF24A82CBB24B2E06B
:101F90002B2E312C2C0E3D1E2E010894411C511C61
:101FA0009E2C812F90E09501281B390BF301E80F3F
:101FB000F91F2530310544F0D10183E001900D92E5
:101FC0008150E1F71D5F09C080819181A281B381B9
:101FD00089839A83AB83BC831C5F892D880FA601FC
:101FE000B201800F0E94630C282F8823E1F4392D61
:101FF0003F5FF601808182FF0EC0812F90E0019645
:102000008A159B0544F40894E11CF11C03E9F3E0F4
:10201000EF16F10429F6181529F4333021F4F601EE
:10202000808182FD2AE0822F90E024960FB6F894FA
:10203000DEBF0FBECDBFDF91CF911F910F91FF90FB
:10204000EF90DF90CF90BF90AF909F908F907F9058
:102050006F905F904F903F902F9008952F923F92F6
:102060004F925F927F928F929F92AF92BF92CF9248
:10207000DF92EF92FF920F931F93CF93DF93982EEF
:10208000EB015A0119016801F80110820E947E06D5
:10209000F82E882309F077C0BE0186E20E94D90E8F
:1020A000F82E882309F06FC0888190E08F719070BE
:1020B000892B19F48FE1F82E66C0F1E09F1689F0A4
:1020C0009F1668F082E0981631F093E0991629F097
:1020D00005E2F02E58C084E905C088E903C083E911
:1020E00001C082E97724882421010894411C511CF5
:1020F000E72CEE0CE80E082D10E0E101C00FD11F17
:10210000AE0160E08E2D0E940E0DF82E8823D9F5C9
:10211000A501BE018E2D0E94630CF82E882399F52F
:102120007394F501808182FF0EC0040D151D43E0FC
:1021300050E0B801CE010E94D721F3E08F0EF601E6
:1021400080818D5F17C0F4E08F0EF60180818C5F77
:1021500011C083E9F3E07F1659F6F501808182FF13
:1021600004C0F601108213E2F12E692D892D0E9420
:102170006F0609C08083F501808182FDEACFF3E01C
:102180007F1699F7EACF8F2D90E0DF91CF911F91C5
:102190000F91FF90EF90DF90CF90BF90AF909F9006
:1021A0008F907F905F904F903F902F900895DC012B
:1021B00070E020E030E011C0E199FECFC901840F4A
:1021C000951F9FBB8EBBFD01E20FF31F80818DBB6E
:1021D000E29AE19A7F5F2F5F3F4F761769F7089584
:1021E000DC01E199FECF70E020E030E00EC0C901D3
:1021F000840F951F9FBB8EBBE09AFD01E20FF31F7A
:102200008DB380837F5F2F5F3F4F761781F70895EF
:10221000E199FECF8EBB6DBBE29AE19A0895E199F8
:10222000FECF8EBBE09A8DB390E008956BE481E120
:102230000E9404016FE382E10E94040161E183E1F5
:102240000E9404016FE284E10E9404016FE385E1D2
:102250000E9404016FE386E10E9404016BE889E1BA
:102260000E94040164E18AE10E9404016DEB8BE1AC
:102270000E9404016FEF8CE10E94040160E08DE197
:102280000E94040161E08EE10E94040160E082E2AC
:102290000E94040162E183E20E94040160EE84E294
:1022A0000E94040180E090E008956BE481E10E94C7
:1022B00004016FE382E10E94040162E083E10E9475
:1022C00004016CE284E10E9404016FE385E10E9455
:1022D00004016FE386E10E9404016FE386E10E943E
:1022E000040160E087E10E9404016BE889E10E943B
:1022F000040160E08AE10E94040162E58BE10E9432
:10230000040166E68CE10E94040160E08DE10E9418
:10231000040161E08EE10E9404016CE082E20E940F
:1023200004016EEF83E20E9404016FEF84E20E94D9
:10233000040180E090E008956BE481E10E940401D3
:102340006FE382E10E94040163E083E10E940401E3
:102350006BE284E10E9404016FE385E10E940401C5
:102360006FE386E10E94040160E087E10E940401BE
:102370006BE889E10E94040164E18AE10E940401A2
:1023800060EE8BE10E9404016FEF8CE10E9404017A
:1023900060E08DE10E94040161E48EE10E9404018D
:1023A0006CE282E20E9404016FEF83E20E9404016A
:1023B0006FEF84E20E94040180E090E00895282FEE
:1023C000E2EFF2E090E003C08FEF81939F5F9217FE
:1023D000D9F70895089508951FBC85E08EBD88E162
:1023E0009EEF9DBD8CBD18BE84E089BF0895292F46
:1023F000332720BD89B982E08BB988E98AB986E89C
:1024000080BD0895823081F0833028F4882341F024
:10241000813071F407C0833059F0843049F406C02C
:102420008FEC07C087E605C084E403C082E201C0E8
:1024300083E389B908955D9BFECF8CB908955F9BB6
:10244000FECF8CB190E008958F708A3020F08950D3
:10245000806490E00895806390E0089582958F7085
:102460000E94241290E00895A2EFB2E0FD010190D5
:102470000020E9F73197EA1BFB0BF0E0EA0FFB1FA6
:1024800005C08C915D9BFECF8CB91196AE17BF072E
:10249000C1F70895C19864E670E080E090E00E9482
:1024A0008E00C19A64E670E080E090E00E948E00A9
:1024B000C19862E370E080E090E00E948E00C19AD3
:1024C00064E670E080E090E00E948E000895C1987C
:1024D00062E370E080E090E00E948E00C19AC198B3
:1024E00062E370E080E090E00E948E00C19A08955F
:1024F000C19868EE73E080E090E00E948E00C19A7F
:102500000895C1989AE0899FC0011124AA2797FDD8
:10251000A095BA2FBC01CD010E948E00C19A0895EA
:10252000C19864E670E080E090E00E948E00C19A5D
:1025300008951F93CF93DF93182F1092E5022091F7
:10254000E202A2EFB2E0922FE92FF0E0EC55FD4F4E
:1025500080818D939F5F83E0A230B807A9F7205F49
:102560002093E202ED016097BE01812F0E948F0A45
:1025700080933C03882331F489E980933C0389E903
:1025800090E009C08091E502882371F785EA809385
:102590003C0385EA90E0DF91CF911F9108951F934E
:1025A000CF93DF93182F1092E5022091E202A2EF61
:1025B000B2E0922FE92FF0E0EC55FD4F80818D9332
:1025C0009F5F83E0A230B807A9F7205F2093E20263
:1025D000ED016097BE01812F0E948F0A80933C031A
:1025E000882331F489E980933C0389E990E009C0AC
:1025F0008091E502882371F785EA80933C0385EAA0
:1026000090E0DF91CF911F9108951F93CF93DF93B7
:10261000182F1092E5022091E202A2EFB2E0922F71
:10262000E92FF0E0EC55FD4F80818D939F5F83E0B3
:10263000A230B807A9F7205F2093E202ED0160976E
:10264000BE01812F0E948F0A80933C03882331F4BE
:1026500089E980933C0389E990E009C08091E50213
:10266000882371F785EA80933C0385EA90E0DF9147
:10267000CF911F9108950F931F93082F162F6CED84
:1026800072E086E20E94D90E882319F566E373E0B2
:1026900080E00E94D20E8823E1F466EE72E086E3C9
:1026A00093E00E94070D8823A1F4212F4AE253E012
:1026B00066E373E080E60E94EE08882351F462EF3F
:1026C00072E0802F0E948F0A882319F40E94DA0595
:1026D00080E090E01F910F9108951F93CF93DF93B7
:1026E000182F1092E502C2EFD2E0BE01812F0E94A6
:1026F0005B0C80933C038823C9F42091E202A2EF93
:10270000B2E0922FE92FF0E0EC55FD4F8D918083E0
:102710009F5F83E0A230B807A9F7205F2093E20211
:1027200089E980933C0389E990E009C08091E50242
:102730008823D9F685EA80933C0385EA90E0DF910F
:10274000CF911F9108951F93CF93DF93182F10926D
:10275000E502C2EFD2E0BE01812F0E945B0C8093A4
:102760003C038823C9F42091E202A2EFB2E0922F49
:10277000E92FF0E0EC55FD4F8D9180839F5F83E062
:10278000A230B807A9F7205F2093E20289E980937D
:102790003C0389E990E009C08091E5028823D9F6DD
:1027A00085EA80933C0385EA90E0DF91CF911F9109
:1027B00008951F93CF93DF93182F1092E502C2EF75
:1027C000D2E0BE01812F0E945B0C80933C038823E2
:1027D000C9F42091E202A2EFB2E0922FE92FF0E0DB
:1027E000EC55FD4F8D9180839F5F83E0A230B80749
:1027F000A9F7205F2093E20289E980933C0389E9ED
:1028000090E009C08091E5028823D9F685EA80939B
:102810003C0385EA90E0DF91CF911F910895DF920C
:10282000EF92FF920F931F93CF93DF93D82E062F33
:102830007A010E94E20614E6CCEDD2E0BE0182E508
:102840000E94D90E80933C03882321F0115009F493
:102850004DC0F4CF66E373E080E00E94D20E90E0BA
:10286000882309F491E090933C03992309F446C02E
:1028700066EE72E086E393E00E94070D90E0882305
:1028800009F491E090933C039923C1F11D2D110FA0
:10289000110F002349F4212F2D5F4D2D66E373E0C6
:1028A00081E60E9469080BC0013059F4212F2D5F89
:1028B00048EF51E066E373E081E60E94EE08809302
:1028C0003C03B701812F8D5F0E948F0A90E088231F
:1028D00009F491E090933C03992381F00E94DD0676
:1028E00089E980933C0389E990E008C00E94DD06F5
:1028F00085EA80933C0385EA90E000C0DF91CF91A8
:102900001F910F91FF90EF90DF900895CF92DF928B
:10291000EF92FF920F931F93CF93DF93CDB7DEB764
:1029200060970FB6F894DEBF0FBECDBFC82ED62E6F
:10293000CA0179016AE273E00E94770420E030E086
:10294000AE014F5F5F4FFA01E20FF31FD701A20FF5
:10295000B31F8C9180832F5F3F4F2630310599F74D
:1029600088E08F8387E788878FE889871A86D80170
:102970009AE0AE014F5F5F4FFA01E90FF11D8D91B3
:1029800080839F5F9031C1F76D2D8C2D0E940F14B5
:1029900080933C03893919F489E990E005C087EAFE
:1029A00080933C0387EA90E060960FB6F894DEBF10
:1029B0000FBECDBFDF91CF911F910F91FF90EF9090
:1029C000DF90CF900895FF920F931F93CF93DF93E3
:1029D000082FF62E0E94E20614E6CCEDD2E0BE01EE
:1029E00086E20E94D90E882321F0115009F443C0D9
:1029F000F6CF66E373E080E00E94D20E882309F0F0
:102A00003FC066EE72E086E393E00E94070D8823E4
:102A1000B9F5102F110F110FFF2049F4212F2D5F51
:102A2000402F66E373E081E60E9469080CC081E0F4
:102A3000F81649F4212F2D5F48EF51E066E373E06B
:102A400081E60E94EE08002329F0812F0E940513E1
:102A50008939B1F4812F8F5F0E94CF12893981F4B7
:102A6000812F8E5F0E949912893951F40E94DD06F0
:102A700089E990E005C00E94DD0685EA90E000C08B
:102A8000DF91CF911F910F91FF900895FF920F93C7
:102A90001F93CF93DF93F82E062F0E94E20614E6D1
:102AA000CCEDD2E0BE0182E50E94D90E882321F050
:102AB000115009F43FC0F6CF66E373E080E00E9456
:102AC000D20E8823E1F566EE72E086E393E00E9481
:102AD000070D8823A1F51F2D110F110F002349F4B5
:102AE000212F2D5F4F2D66E373E080E60E94690879
:102AF0000BC0013049F4212F2D5F46E152E066E31F
:102B000073E080E60E94EE08812F0E94D913893974
:102B1000B1F4812F8F5F0E94A313893981F4812F33
:102B20008E5F0E946D13893951F40E94DD0689E998
:102B300090E005C00E94DD0685EA90E000C0DF91CC
:102B4000CF911F910F91FF9008951F93CF93DF9323
:102B5000E2EFF2E08FEF819383E0E230F807D1F704
:102B60000E94E2061AE0CCEDD2E0BE0182E50E94AE
:102B7000D90E80933C03882319F01150E1F0F5CF72
:102B800066E373E080E00E94D20E80933C038823CA
:102B9000D1F466EE72E086E393E00E94070D809325
:102BA0003C03882381F40E94DD0689E980933C037D
:102BB00089E990E008C00E94DD0685EA80933C0325
:102BC00085EA90E000C0DF91CF911F9108956F9248
:102BD0007F928F929F92AF92BF92CF92DF92EF92AD
:102BE000FF920F931F93CF93DF934C0160E070E04F
:102BF00036E0632E712CF4012281273309F440C0A2
:102C0000283380F4233381F1243338F4213331F134
:102C1000223338F52033E1F41EC0253359F1263331
:102C200060F525C02236C1F1233638F4293371F11D
:102C3000293348F1213661F42CC0243699F1243629
:102C400070F1253691F1263619F4CFE0D0E02FC08F
:102C5000CFEFD0E02CC0C0E0D0E029C0C1E0D0E090
:102C600026C0C2E0D0E023C0C3E0D0E020C0C4E072
:102C7000D0E01DC0C5E0D0E01AC0C6E0D0E017C06B
:102C8000C7E0D0E014C0C8E0D0E011C0C9E0D0E097
:102C90000EC0CAE0D0E00BC0CBE0D0E008C0CCE072
:102CA000D0E005C0CDE0D0E002C0CEE0D0E0882783
:102CB00077FD8095982F0E94801F5B016C01B30106
:102CC000882777FD8095982F0E94801F9B01AC017B
:102CD00060E070E080E891E40E944E227B018C016C
:102CE000BE01882777FD8095982F0E94801F9B0149
:102CF000AC01C801B7010E94811E9B01AC01C60155
:102D0000B5010E94541E0E94DE1F0894811C911C74
:102D10006114710421F00894610871086CCF5D9B07
:102D2000FECF6CB9DF91CF911F910F91FF90EF9083
:102D3000DF90CF90BF90AF909F908F907F906F90DB
:102D4000089520E030E0FC01E20FF31FE0815D9B7D
:102D5000FECFECB92F5F3F4F20323105A1F75D9BCD
:102D6000FECF8DE08CB95D9BFECF8AE08CB90895D3
:102D7000AF92BF92CF92DF92EF92FF920F931F9389
:102D8000CF93DF939FEF9BBB9ABB8EEA88BB8AEA07
:102D900087BB95BB94BB80E382BB8CE381BB0E9465
:102DA000901268EE73E080E090E00E948E0068EE82
:102DB00073E080E090E00E948E008BB78F7D8BBF28
:102DC00084B784BF8BB78F7B8BBF8BB78F778BBF5D
:102DD000579889B78B7F89BF8BB780628BBF7894F8
:102DE000479A0E94C7000E94E000C49A0E94EC111A
:102DF0000E9475070E94CA0680E190E00E94F711C8
:102E000083E08093E4020E94021289E10E941B0188
:102E100089E10E941B0165EA70E082EF92E00E9466
:102E2000E92182EF92E00E943412579A89B78B7F92
:102E300089BF1092E3020E94DD060E94781281E0B1
:102E40008093DE020E94E2060E94A515893969F589
:102E50008AE00E9481125D9BFECF8BEF8CB95D9B57
:102E6000FECF81E08CB9909139035D9BFECF9CB978
:102E7000809138035D9BFECF8CB9309137035D9B09
:102E8000FECF3CB9209136035D9BFECF2CB998272D
:102E900081E0982793279227909329035D9BFECF8B
:102EA0009CB95D9BFECF8CEF8CB98091DE028823AC
:102EB00059F6C4EAD2E062EFE62E62E0F62E5DE358
:102EC000A52E53E0B52E4AEEC42E42E0D42E8091BA
:102ED000E302813009F048C0109229031092E30206
:102EE0000E94A515893949F55D9BFECF8BEF8CB902
:102EF0005D9BFECF81E08CB9909139035D9BFECF45
:102F00009CB9809138035D9BFECF8CB9309137031B
:102F10005D9BFECF3CB9209136035D9BFECF2CB963
:102F2000982781E0982793279227909329035D9B08
:102F3000FECF9CB95D9BFECF15C05D9BFECF8BEF96
:102F40008CB95D9BFECF81E08CB95D9BFECF85EA9D
:102F50008CB984EA809329035D9BFECF84EA8CB907
:102F60005D9BFECF8CEF8CB98091E302823009F03B
:102F70005BC01092290385E08093E9021092E3027E
:102F80001092E2026091F1028091F0020E944615D7
:102F9000893989F5109229035D9BFECF8BEF8CB99F
:102FA0005D9BFECF82E08CB9809329039091F00263
:102FB0005D9BFECF9CB982E08927809329032091F5
:102FC000E7025D9BFECF2CB9822780932903FE0187
:102FD00030E007C090815D9BFECF9CB989273F5FA1
:102FE00031963217B9F7809329035D9BFECF8CB9D8
:102FF0005D9BFECF17C05D9BFECF8BEF8CB95D9BB9
:10300000FECF82E08CB95D9BFECF85EA8CB99091B2
:10301000290387EA9827909329035D9BFECF9CB9EB
:103020005D9BFECF8CEF8CB98091E302843009F078
:103030003FC0109229031092E3021092E2026091C5
:10304000F1028091F0020E94E3148939C1F45D9B82
:10305000FECF8BEF8CB95D9BFECF84E08CB95D9B7E
:10306000FECF89E98CB9909129038DE99827909337
:1030700029035D9BFECF9CB95D9BFECF17C05D9B76
:10308000FECF8BEF8CB95D9BFECF84E08CB95D9B4E
:10309000FECF85EA8CB99091290381EA9827909315
:1030A00029035D9BFECF9CB95D9BFECF8CEF8CB955
:1030B0008091E302853009F085C0109229031092B7
:1030C000E3028091A402F701819393E0E232F907D1
:1030D000D9F78091F0028F3FF1F500E010E06091A8
:1030E000F102802F0E94E3140F5F1F4F0031110582
:1030F000B1F78939C1F45D9BFECF8BEF8CB95D9B35
:10310000FECF85E08CB95D9BFECF89E98CB99091AB
:1031100029038CE99827909329035D9BFECF9CB9E6
:103120005D9BFECF4DC05D9BFECF8BEF8CB95D9B51
:10313000FECF85E08CB95D9BFECF85EA8CB990917E
:10314000290380EA9827909329035D9BFECF9CB9C1
:103150005D9BFECF35C06091F1020E94E314893976
:10316000C1F45D9BFECF8BEF8CB95D9BFECF85E0FC
:103170008CB95D9BFECF89E98CB9909129038CE9CC
:103180009827909329035D9BFECF9CB95D9BFECF52
:1031900017C05D9BFECF8BEF8CB95D9BFECF85E0AA
:1031A0008CB95D9BFECF85EA8CB99091290380EAAA
:1031B0009827909329035D9BFECF9CB95D9BFECF22
:1031C0008CEF8CB98091E3028A3009F079C01092BB
:1031D00029031092E3028091DF028036B9F56091F5
:1031E000F002AE010E9453058823C1F45D9BFECF1F
:1031F0008BEF8CB95D9BFECF8AE08CB95D9BFECFD7
:1032000089E98CB99091290383E998279093290340
:103210005D9BFECF9CB95D9BFECF50C05D9BFECFFA
:103220008BEF8CB95D9BFECF8AE08CB95D9BFECFA6
:1032300087EA8CB9909129038DEA98279093290306
:103240005D9BFECF9CB95D9BFECF38C08136C1F53A
:103250006091F002AE010E9453058823C1F45D9B8A
:10326000FECF8BEF8CB95D9BFECF8AE08CB95D9B66
:10327000FECF89E98CB99091290383E9982790932F
:1032800029035D9BFECF9CB95D9BFECF17C05D9B64
:10329000FECF8BEF8CB95D9BFECF8AE08CB95D9B36
:1032A000FECF87EA8CB9909129038DEA98279093F5
:1032B00029035D9BFECF9CB95D9BFECF8CEF8CB943
:1032C0008091E3028A3409F075C0109229031092AC
:1032D000E3028091DF028036A9F5BE010E949C04C2
:1032E0008823C1F45D9BFECF8BEF8CB95D9BFECF35
:1032F0008AE48CB95D9BFECF89E98CB99091290352
:1033000083ED9827909329035D9BFECF9CB95D9B2D
:10331000FECF4EC05D9BFECF8BEF8CB95D9BFECF89
:103320008AE48CB95D9BFECF87EA8CB99091290322
:103330008DEE9827909329035D9BFECF9CB95D9BF2
:10334000FECF36C08136B1F5BE010E949C048823B1
:10335000C1F45D9BFECF8BEF8CB95D9BFECF8AE401
:103360008CB95D9BFECF89E98CB99091290383EDDF
:103370009827909329035D9BFECF9CB95D9BFECF60
:1033800017C05D9BFECF8BEF8CB95D9BFECF8AE0B3
:103390008CB95D9BFECF87EA8CB9909129038DEAA9
:1033A0009827909329035D9BFECF9CB95D9BFECF30
:1033B0008CEF8CB98091E3028A3309F088CD1092AA
:1033C00029031092E3026091F10285019601A701A1
:1033D0008091F0020E9486148939C1F45D9BFECF72
:1033E0008BEF8CB95D9BFECF8AE38CB95D9BFECFE2
:1033F00089E98CB99091290383EA9827909329034E
:103400005D9BFECF9CB95D9BFECF17C05D9BFECF41
:103410008BEF8CB95D9BFECF8AE38CB95D9BFECFB1
:1034200087EA8CB9909129038DE998279093290315
:103430005D9BFECF9CB95D9BFECF8CEF8CB947CDD9
:103440001F920F920FB60F9211242F933F934F9319
:103450005F936F937F938F939F93AF93BF93EF93FC
:10346000FF931092E3025F9BFECF8CB190E08B3F05
:1034700009F491E09093D902992309F432C25F9B39
:10348000FECF8CB18093E802882329F55F9BFECFA5
:103490008CB190E08C3F09F491E09093E102992384
:1034A00089F00E9490121092DE025D9BFECF8BEF9E
:1034B0008CB95D9BFECF81E08CB95D9BFECF8CEF1C
:1034C0008CB909C01092F0021092E7028FEF80933E
:1034D000E8021092E3028091E802813091F45F9B50
:1034E000FECF8CB1809329035F9BFECF8CB190E01F
:1034F0008C3F09F491E09093E102992381F181E0FE
:1035000022C0823061F55F9BFECF8CB18093F002C8
:103510005F9BFECF8CB18093F1025F9BFECF8CB19D
:103520008093E7025F9BFECF8CB1809329035F9B62
:10353000FECF8CB190E08C3F09F491E09093E102D2
:10354000992321F082E08093E30209C01092F002F7
:103550001092E7028FEF8093E8021092E3028091CD
:10356000E8028430E9F55F9BFECF8CB18093F002D6
:103570005F9BFECF8CB18093F1025F9BFECF2CB19D
:103580002093E702A4EAB2E0FD01119282E0E43D5B
:10359000F807D9F790E005C05F9BFECF8CB18D9303
:1035A0009F5F9217C9F75F9BFECF8CB18093290371
:1035B0005F9BFECF8CB190E08C3F09F491E090933B
:1035C000E102992321F084E08093E30209C0109284
:1035D000F0021092E7028FEF8093E8021092E3026C
:1035E0008091E802853051F55F9BFECF8CB18093CE
:1035F000F0025F9BFECF8CB18093F1025F9BFECF08
:103600008CB18093A4025F9BFECF8CB18093290381
:103610005F9BFECF8CB190E08C3F09F491E09093DA
:10362000E102992321F085E08093E30207C08FEF48
:103630008093F0028093E8021092E3028091E80206
:103640008A30C9F55F9BFECF8CB18093F0025F9BFF
:10365000FECF2CB12093E702E4EAF2E090E005C04F
:103660005F9BFECF8CB181939F5F9217C9F75F9BE1
:10367000FECF8CB18093DF025F9BFECF8CB1809335
:1036800029035F9BFECF8CB190E08C3F09F491E061
:103690009093E102992321F08AE08093E3020BC02A
:1036A0001092DF021092F0021092E7028FEF8093E7
:1036B000E8021092E3028091E8028A3491F55F9B60
:1036C000FECF2CB12093E702E4EAF2E090E005C0DF
:1036D0005F9BFECF8CB181939F5F9217C9F75F9B71
:1036E000FECF8CB18093DF025F9BFECF8CB18093C5
:1036F00029035F9BFECF8CB190E08C3F09F491E0F1
:103700009093E102992321F08AE48093E30209C0B7
:103710001092DF021092E7028FEF8093E80210927E
:10372000E3028091E8028A3109F055C05F9BFECF29
:103730008CB18093E4025F9BFECF8CB18093290310
:103740005F9BFECF8CB190E08C3F09F491E09093A9
:10375000E1029923B9F10E9490128091E4028093D2
:10376000F20246E151E061E082EF92E00E94D71060
:103770005D9BFECF8BEF8CB95D9BFECF8AE18CB950
:103780009091E4025D9BFECF9CB95D9BFECF8AE1E8
:1037900098279CB95D9BFECF8CEF8CB946E151E038
:1037A00061E082EF92E00E94F0108091F20280933B
:1037B000E40280E190E00E94F7118091E4020E940F
:1037C000021209C01092F0021092E7028FEF80936C
:1037D000E8021092E3028091E8028A32C1F55F9B11
:1037E000FECF2CB120933B035F9BFECF8CB1809327
:1037F00029035F9BFECF8CB190E08C3F09F491E0F0
:103800009093E1029923D1F0822F0E9481125D9B57
:10381000FECF8BEF8CB95D9BFECF8AE28CB9809195
:103820003B035D9BFECF8CB9809129035D9BFECF4E
:103830008CB95D9BFECF8CEF8CB909C01092F00261
:103840001092E7028FEF8093E8021092E3028091DA
:10385000E8028A3309F045C05F9BFECF8CB18093AC
:10386000F0025F9BFECF8CB18093F102E2EFF2E0B9
:103870005F9BFECF8CB1819382E0E83FF807C1F7F0
:10388000EAEEF2E05F9BFECF8CB1819382E0E03FF5
:10389000F807C1F7EDE3F3E05F9BFECF8CB18193B6
:1038A00083E0E334F807C1F75F9BFECF8CB18093D0
:1038B00029035F9BFECF8CB190E08C3F09F491E02F
:1038C0009093E102992321F08AE38093E30209C0F7
:1038D0001092F0021092E7028FEF8093E8021092AC
:1038E000E302FF91EF91BF91AF919F918F917F91F3
:1038F0006F915F914F913F912F910F900FBE0F905D
:103900001F9018951F920F920FB60F9211248F934C
:103910009F9387EF92EC9DBD8CBD8091E902815011
:103920008093E902882311F41092E5029F918F9110
:103930000F900FBE0F901F9018950F931F93CF936A
:10394000DF93082F162FC2EFD2E08FEF899383E029
:10395000C230D807D1F76CED72E086E20E94D90E32
:10396000882319F083E090E023C066E373E080E0F1
:103970000E94D20E8823C9F466EE72E086E393E0DB
:103980000E94070D882389F4212F4AE253E066E361
:1039900073E080E60E94EE08882339F4BE0160518E
:1039A0007040802F0E945B0C811102C080E090E08B
:1039B000DF91CF911F910F910895A0E0B0E0E3EE69
:1039C000FCE10C9419222C015B01FA01DC019C91B1
:1039D000923008F432C1EB018881823008F42CC1A6
:1039E000943071F4843009F028C1F2019181898109
:1039F000981709F422C11DED412E10E0512E1DC172
:103A0000843009F419C18230A9F4923009F015C14B
:103A1000CA01A20128E0DA010D90AD01EC01099282
:103A2000CE012150C1F7E5018981E2019981892305
:103A3000818300C1923009F4FFC0E201CA80DB80BB
:103A4000EB018A819B81E2012C813D814E815F8166
:103A5000EB01EC80FD800E811F81B601681B790BA4
:103A6000DB0177FF03C0709561957F4F6032710570
:103A70000CF05DC01A161B065CF566247724430122
:103A800081E090E0A0E0B0E0062E04C0880F991F0E
:103A9000AA1FBB1F0A94D2F70197A109B1098E2171
:103AA0009F21A023B1230097A105B10529F0B1E022
:103AB0006B2E712C812C912C04C016950795F794D0
:103AC000E7946A95D2F7E628F728082919293BC018
:103AD000AB2BC9F1C60ED71E66247724430181E0C3
:103AE00090E0A0E0B0E0062E04C0880F991FAA1F46
:103AF000BB1F0A94D2F70197A109B109822393232E
:103B0000A423B5230097A105B10529F0A1E06A2EF1
:103B1000712C812C912C04C056954795379527958B
:103B20006A95D2F726293729482959290CC08C15BE
:103B30009D0534F06C0120E030E040E050E003C02F
:103B4000EE24FF248701E2019981E501898198171C
:103B500009F443C0992339F0E21AF30A040B150B58
:103B6000A801970104C02E193F09400B510B57FDC6
:103B700008C01182D382C28224833583468357834F
:103B80001DC081E08183D382C28288279927DC010E
:103B9000821B930BA40BB50B84839583A683B783F9
:103BA0000DC0220F331F441F551F248335834683C6
:103BB0005783828193810197938382832481358106
:103BC00046815781DA01C9010197A109B1098F5FC7
:103BD0009F4FAF4FBF4328F30BC09183D382C28264
:103BE0002E0D3F1D401F511F24833583468357836D
:103BF00083E0808324813581468157815523D4F425
:103C0000C901AA2797FDA095BA2F81709070A07066
:103C1000B0705695479537952795822B932BA42BFB
:103C2000B52B84839583A683B78382819381019684
:103C3000938382832F0101C02501C201E0E1CDB74A
:103C4000DEB70C943522A0E2B0E0E9E2FEE10C948C
:103C5000232269837A838B839C832D833E834F83C6
:103C6000588709E0E02EF12CEC0EFD1EB701CE01C5
:103C700001960E945E218E010F5E1F4FB801CE019A
:103C800005960E945E218A8991E089278A8BAE0180
:103C9000475E5F4FB801C7010E94DD1C0E947E2075
:103CA000E6E0A0960C943F22A0E2B0E0EAE5FEE157
:103CB0000C94232269837A838B839C832D833E8398
:103CC0004F83588789E0E82EF12CEC0EFD1EB701DA
:103CD000CE0101960E945E218E010F5E1F4FB8013A
:103CE000CE0105960E945E21AE01475E5F4FB8018E
:103CF000C7010E94DD1C0E947E20E6E0A0960C9485
:103D00003F22A0E2B0E0E7E8FEE10C9419226983CB
:103D10007A838B839C832D833E834F83588799E0DE
:103D2000E92EF12CEC0EFD1EB701CE0101960E948A
:103D30005E218E010F5E1F4FB801CE0105960E94D5
:103D40005E219985923088F089898230C0F0943064
:103D500019F4823029F009C0843029F4923079F4C2
:103D60006DED70E0C6C0923041F420E09A858A89FA
:103D7000981321E02A87B701BCC0823041F420E0CB
:103D80009A858A89981321E02A8BB801B2C0CD8424
:103D9000DE84EF84F8880D891E892F89388D882468
:103DA0009924540140E050E060E070E04424552440
:103DB0003201E0E0F0E0C60181709070892BD9F00B
:103DC000800E911EA21EB31EDB01CA01840D951D3B
:103DD000A61DB71D40E050E060E070E0801691063F
:103DE000A206B30620F441E050E060E070E0480F26
:103DF000591F6A1F7B1F440C551C661C771C37FF1C
:103E000008C081E090E0A0E0B0E0482A592A6A2A80
:103E10007B2A3196E032F10549F0000F111F221F75
:103E2000331FF694E794D794C794C5CF8B899C89A8
:103E30002B853C85820F931F02969C8F8B8F1A8E49
:103E40009A858A89981711F081E08A8F2B8D3C8D95
:103E500017C0CA0181709070892B61F0B694A79445
:103E60009794879480E090E0A0E0B0E8882A992AAF
:103E7000AA2ABB2A76956795579547952F5F3F4F9E
:103E800077FDE7CFC9010BC0440F551F661F771F91
:103E9000B7FC4160880C991CAA1CBB1C01974030E0
:103EA000A0E05A07A0E06A07A0E47A0768F39C8FB5
:103EB0008B8FDB01CA018F779070A070B070803457
:103EC0009105A105B10561F447FD0AC08114910473
:103ED000A104B10429F0405C5F4F6F4F7F4F4078E1
:103EE0004D8F5E8F6F8F78A383E0898FBE01675EF1
:103EF0007F4FCB010E947E20E0E1A0960C943522FA
:103F0000A8E0B0E0E6E8FFE10C9420229B01AC01C0
:103F100083E08983DA01C9018827B7FD8395992752
:103F2000AA27BB27B82E211531054105510519F4E3
:103F300082E089833AC08823A9F0203080E03807E6
:103F400080E0480780E8580729F460E070E080E0EE
:103F50009FEC30C0EE24FF248701E21AF30A040B21
:103F6000150B02C079018A018EE1C82ED12CDC82AA
:103F7000CB82ED82FE820F831887C801B7010E94B1
:103F8000312001971816190684F4082E04C0EE0C8F
:103F9000FF1C001F111F0A94D2F7ED82FE820F83CF
:103FA0001887C81AD90ADC82CB82BA82CE01019660
:103FB0000E947E20E9E028960C943C22ACE0B0E020
:103FC000E4EEFFE10C94272269837A838B839C8340
:103FD000BE016B5F7F4FCE0101960E945E218D81F5
:103FE0008230A9F1823098F1843021F48E818823C7
:103FF00059F40FC02F81388537FD29C06E812F31CC
:10400000310564F0662329F020E030E040E050E81C
:1040100022C02FEF3FEF4FEF5FE71DC08EE190E032
:10402000821B930B29853A854B855C8504C0569588
:104030004795379527958A95D2F7662361F0509575
:104040004095309521953F4F4F4F5F4F04C020E082
:1040500030E040E050E0CA01B901E2E02C960C9457
:104060004322EF92FF920F931F939B01AC012030EC
:1040700080E0380781E0480780E0580780F42F3F50
:1040800031054105510509F020F4EE24FF24870194
:1040900019C068E0E62EF12C012D112D13C020303F
:1040A00080E0380780E0480781E0580730F490E16D
:1040B000E92EF12C012D112D05C088E1E82EF12CFF
:1040C000012D112D80E290E0A0E0B0E08E199F0953
:1040D000A00BB10B04C05695479537952795EA94E8
:1040E000D2F7F901EB51FF4F2081821B9109A10901
:1040F000B1091F910F91FF90EF9008959F92AF9299
:10410000BF92CF92DF92EF92FF920F931F93EE2414
:10411000FF248701FC0124813581468157819180EC
:104120008081823010F44061A2C0843009F49BC0C9
:10413000823029F420E030E040E050E005C0211555
:1041400031054105510519F4E0E0F0E092C08281AB
:1041500093816FEF823896070CF05AC062E87FEFC8
:10416000681B790B6A3171052CF020E030E040E0EB
:1041700050E02AC0AA24BB24650181E090E0A0E0C1
:10418000B0E0062E04C0880F991FAA1FBB1F0A9417
:10419000D2F70197A109B10982239323A423B52360
:1041A0000097A105B10529F071E0A72EB12CC12C13
:1041B000D12C04C056954795379527956A95D2F727
:1041C0002A293B294C295D29DA01C9018F77907092
:1041D000A070B07080349105A105B10539F427FFB6
:1041E00009C0205C3F4F4F4F5F4F04C0215C3F4FE1
:1041F0004F4F5F4F80E090E0203060E0360760E096
:10420000460760E4560710F081E090E0FC0123C00F
:104210008038910544F5FC01E158FF4FDA01C901EE
:104220008F779070A070B07080349105A105B105B2
:1042300039F427FF09C0205C3F4F4F4F5F4F04C048
:10424000215C3F4F4F4F5F4F57FF05C05695479535
:1042500037952795319687E0569547953795279559
:104260008A95D1F706C020E030E040E050E0EFEF63
:10427000F0E0E22EF32E942F9F77802F8078892B09
:104280009E2F9795992797958F77082F092B9E2F0B
:104290009695812F8078892B9794992497948F777E
:1042A000182F1929C801B7011F910F91FF90EF90A6
:1042B000DF90CF90BF90AF909F900895CF93DF9302
:1042C000FC01DB01208131819281492F4F7750E041
:1042D000991F9927991F8381E82FEE0FE92B6E2FE5
:1042E00070E0881F8827881FED018983EE2371F510
:1042F000211531054105510511F482E02FC06E579B
:104300007040FD017383628367E0220F331F441FF7
:10431000551F6A95D1F783E08C930AC0220F331F93
:10432000441F551FED018A819B8101979B838A83DE
:104330002030E0E03E07E0E04E07E0E45E0770F387
:10434000ED012C833D834E835F8325C0EF3F79F4DD
:10435000211531054105510519F484E08C931BC0EA
:1043600044FF03C081E08C9311C01C920FC06F57B3
:104370007040ED017B836A8383E08C9387E0220F9A
:10438000331F441F551F8A95D1F75064FD012483C4
:10439000358346835783DF91CF910895FB01DC017C
:1043A00002C001900D9241505040D8F7089568170F
:1043B000790768F4FB01DC01E40FF51FA40FB51FBA
:1043C00002C002900E9241505040D8F708950C94CC
:1043D000CE21FB01DC0101900D920020E1F7089550
:1043E00097FB092E07260AD077FD04D00CD006D003
:1043F00000201AF4709561957F4F0895F6F7909517
:1044000081959F4F0895AA1BBB1B51E107C0AA1FAE
:10441000BB1FA617B70710F0A61BB70B881F991F65
:104420005A95A9F780959095BC01CD0108952F92DA
:104430003F924F925F926F927F928F929F92AF9234
:10444000BF92CF92DF92EF92FF920F931F93CF9381
:10445000DF93CDB7DEB7CA1BDB0B0FB6F894DEBF18
:104460000FBECDBF09942A88398848885F846E843E
:104470007D848C849B84AA84B984C884DF80EE8088
:10448000FD800C811B81AA81B981CE0FD11D0FB691
:10449000F894DEBF0FBECDBFED010895FA01EE0F17
:1044A000FF1F30962105310599F16115710561F401
:1044B0008038BFE39B0749F168949038810561F02B
:1044C0008038BFEF9B0741F0992342F5FF3FE1059C
:1044D0003105210511F1E8940894E795D901AA2343
:1044E00029F4AB2FBE2FF85FD0F310C0FF5F70F43C
:1044F000A695E0F7F73950F019F0FF3A38F49F77B6
:104500009F930CD00F9007FC905808953EF049C03F
:1045100060E070E080E89FE308954FE79F775F9346
:104520004F933F932F93D0D02F913F914F915F9115
:10453000E8DB05C019F40EF02EC07DC032C061D09A
:10454000C8F39638C0F707F80F92E8942BE33AEADD
:1045500048EB5FE738D10F920F920F924DB75EB7DD
:104560000F92F2D0E4E5F0E01FD04F915F91EF9110
:10457000FF91E595EE1FFF1F49F0FE57E0684427C5
:10458000EE0F441FFA95E1F74195550B64D00F905B
:1045900007FE58C0089597F99F6780E870E060E0D3
:1045A00008959FEF80EC0895DF93CF931F930F93AF
:1045B000FF92EF92DF927B018C01689405C0DA2EA6
:1045C000EF01FFD0FE01E894A59125913591459129
:1045D0005591AEF3EF0159D1FE019701A801DA948C
:1045E00079F7DF90EF90FF900F911F91CF91DF91BE
:1045F000089557FD9058440F551F59F05F3F71F0D3
:104600004795880F97FB991F61F09F3F79F0879539
:104610000895121613061406551FF2CF4695F1DFC2
:1046200008C0161617061806991FF1CF8695710552
:10463000610508940895E894BB2766277727CB0186
:1046400097F908959B01AC0160E070E080E89FE37A
:104650006FC1A1CFD5C1D5DFE8F39923D9F3940F6A
:10466000511DBBF39150504094F059F0882332F023
:10467000660F771F881F91505040C1F79E3F51052C
:1046800044F7880F911D9695879597F908955F3F98
:10469000ACF0983E9CF0BB27869577956795B795CB
:1046A00008F4B1609395C1F7BB0F58F711F460FFA0
:1046B000E8CF6F5F7F4F8F4F9F4FE3CFBDCF0EF09F
:1046C0009FC16FCF689467CF9CDFC8F39923D1F364
:1046D000C6F3DF93CF931F930F93FF92C92FDD276C
:1046E00088232AF02197660F771F881FDAF720E0CA
:1046F00030E040E85FEB9FE3883920F0803E30F007
:1047000021968F77D1DAECE7F0E003C0CDDAE9EA61
:10471000F0E04ADF8B01BE01EC01FB2E6F577109FF
:104720007595771F880B990BEBDB28E132E741E3A6
:104730005FE347D0AF2D9801AE01FF900F911F911D
:10474000CF91DF91A2D07AC1FA01DC01AA0FBB1F81
:104750009B01AC01BF5728F4222733274427507808
:104760001FC0B75188F4AB2F002446953795279585
:10477000011CA395D2F3002069F0220F331F441FC0
:10478000B395DAF30DD05FCA61307105A0E88A07EE
:10479000B94630F49B01AC016627772788279078CB
:1047A000309621F02083318342835383089538D19A
:1047B00028F03DD118F0952309F0EDCEF2CE11246A
:1047C0003BCF17DFA0F3959FD1F3950F50E0551F16
:1047D000629FF001729FBB27F00DB11D639FAA2756
:1047E000F00DB11DAA1F649F6627B00DA11D661FA5
:1047F000829F2227B00DA11D621F739FB00DA11DC6
:10480000621F839FA00D611D221F749F3327A00D7F
:10481000611D231F849F600D211D822F762F6A2F1B
:1048200011249F5750408AF0E1F088234AF0EE0FA0
:10483000FF1FBB1F661F771F881F91505040A9F7AD
:104840009E3F510570F0A7CEF7CE5F3FECF3983E48
:10485000DCF3869577956795B795F795E7959F5F14
:10486000C1F7FE2B880F911D9695879597F90895AE
:10487000D7D030F0DCD020F031F49F3F11F41EF49B
:1048800090CE0EF4E095E7FB86CEE92FB2DE80F302
:10489000BA17620773078407950718F071F49EF53D
:1048A000CACE0EF4E0950B2EBA2FA02D0B01B90144
:1048B00090010C01CA01A0011124FF27591B99F096
:1048C000593F50F4503E68F11A16F040A22F232FA2
:1048D000342F4427585FF3CF469537952795A795F2
:1048E000F0405395C9F77EF41F16BA0B620B730B99
:1048F000840BBAF09150A1F0FF0FBB1F661F771F0A
:10490000881FC2F70EC0BA0F621F731F841F48F4BE
:10491000879577956795B795F7959E3F08F0B3CF44
:104920009395880F08F09927EE0F9795879508952E
:104930000CD084C07CD040F073D030F021F45F3FC5
:1049400019F029CE511178CE2CCE53DE98F399234D
:10495000C9F35523B1F3951B550BBB27AA27621743
:104960007307840738F09F5F5F4F220F331F441F88
:10497000AA1FA9F333D00E2E3AF0E0E830D09150C0
:104980005040E695001CCAF729D0FE2F27D0660FAD
:10499000771F881FBB1F261737074807AB07B0E8EC
:1049A00009F0BB0B802DBF01FF2793585F4F2AF002
:1049B0009E3F510568F0EFCD3FCE5F3FECF3983E50
:1049C000DCF3869577956795B795F7959F5FC9F75F
:1049D000880F911D9695879597F90895E1E0660FE8
:1049E000771F881FBB1F621773078407BA0720F061
:1049F000621B730B840BBA0BEE1F88F7E0950895CA
:104A00009F3F49F0915028F4869577956795B79523
:104A10009F5F80389F4F880F9695879597F90895E7
:104A200000240A941616170618060906089500248D
:104A30000A9412161306140605060895092E039407
:104A4000000C11F4882352F0BB0F40F4BF2B11F47B
:104A500060FF04C06F5F7F4F8F4F9F4F0895FFCF60
:104A60003030303030303030303030303030303046
:104A7000006202620273000800FF00000053000998
:104A80000050000C003300090050000C0013000916
:104A90000050000C0019001300110007000900036A
:104AA000000100010052433533312D484620524663
:104AB000494420526561646572204669726D776170
:104AC00072652056312E33284743432900F8778FEB
:104AD00000F8778F00F8778F00F8778F00000000DC
:104AE00000000000000001020203030303040404A9
:104AF000040404040405050505050505050505056B
:104B0000050505050506060606060606060606064A
:104B10000606060606060606060606060606060635
:104B2000060606060607070707070707070707071A
:104B30000707070707070707070707070707070705
:104B400007070707070707070707070707070707F5
:104B500007070707070707070707070707070707E5
:104B600007070707070808080808080808080808CA
:104B700008080808080808080808080808080808B5
:104B800008080808080808080808080808080808A5
:104B90000808080808080808080808080808080895
:104BA0000808080808080808080808080808080885
:104BB0000808080808080808080808080808080875
:104BC0000808080808080808080808080808080865
:104BD0000808080808080808080808080808080855
:064BE000080808080800A7
:00000001FF
